:2000000093CA15C0EBCA13C012C011C010C00FC00EC00DC00CC00BC00AC009C008C0112422
:200020001FBECFE5D2E0DEBFCDBF02D002C0E8CFFFCFF89400C0F894FFCF00000000000095
:20148000FFFFFFFFFFFFFFFFFFFFFFFFFFFFFFFFFFFFFFFFFFFFFFFFFFFFFFFFFFFFFFFF6C
:2014A000FFFFFFFFFFFFFFFFFFFFFFFFFFFFFFFFFFFFFFFFFFFFFFFFFFFFFFFFB8C5AFC557
:2014C00033C05FC08BC05DC05CC05BC05AC059C058C057C056C055C054C053C052C009028A
:2014E0001200010100803209040000000000000012011001FF00000881179F0C05010102A2
:20150000000110035400720069006E006B006500740012034100640061006600720075006E
:20152000690074000403090411241FBECFE5D2E0DEBFCDBF84B7877F84BF88E10FB6F894DB
:2015400081BD11BC0FBE91E080E80FB6F89486BD96BD0FBE0AEA0F9310E0A0E6B0E0EEEDAF
:20156000FFE102C005900D92A236B107D9F711E0A2E6B0E001C01D92A832B107E1F7F2D38D
:201580002CC59ECFA82FB92F80E090E041E050EA609530E009C02D9182279795879510F086
:2015A00084279527305EC8F36F5FA8F30895EADF8D939D930895A6E088279927AA9569F032
:2015C0000197E1F3B399FCCFB39BFECF81E09927A6B3019611F0A871D9F70895CF93CFB7ED
:2015E000CF93C0915F02CA3A21F0CF91CFBFCF9165CFCC27C395B39BE9F7B39B0BC0B39B60
:2016000009C0B39B07C0B39B05C0B39B03C0B39B01C0D3C00F92DF93C0910B01DD27CE5E86
:20162000DE4F012EB39B03C0DF910F90E6CF2F930F931F934F932FEF4F6F06B303FB20F9D5
:201640005F933F9350E03BE065C016B30126502953FDC89556B3012703FB25F92F7306B398
:20166000B1F05027102713FB26F906B22230F0F000C016B3012703FB27F90126502906B2DD
:201680002430E8F54F77206816B30000F6CF50274F7D206206B2102F000000C006B30026E2
:2016A0005029102713FB26F906B2E2CF4F7B06B3206400C0DACF01265029187106B269F139
:2016C0004E7F2160012F16B328C0002650294D7F06B22260102F29C0012650294B7F06B2EC
:2016E0002460012F2DC016B301265029477F2860000006B22EC04F7E06B3206130C042278C
:2017000006B3499300265029102706B24FEF13FB20F9297F16B379F2187159F101265029F2
:2017200006B2012703FB21F9237F06B371F2002650293150D0F006B2102713FB22F9277E56
:2017400016B351F201265029012703FB06B223F92F7C49F2000006B3102713FB24F90026BC
:20176000502906B22F7939F270CF10E21ABF002717C03B503195C31BD04010E21ABF0881CA
:20178000033CF9F00B34E9F0209109011981110F1213EDCF093651F10D3211F0013E39F783
:2017A000009310013F915F914F911F910F912F91DF910F90CAB7C5FD1DCFCF91CFBFCF9149
:2017C000189520911001222369F310910E01112321F5343022F130930E0120930A01109157
:2017E0000B013BE0311B30930B0119C000910E0101309CF40AE53091600034FD11C00093C8
:201800006000CEEFD0E010C0052710E000C021C0052710E0C89508BB14C03AE501C032ED5F
:20182000032EC0E0D0E032E017B31861C39A08B317BB58E120E84FEF20FF052708BB27959F
:2018400017951C3F28F700004552B0F720FF0527279508BB17951C3FB8F629913A9561F7C4
:20186000077E10910F01110F08BBC250D04011F01093090110E21ABF086017B3177E402F7E
:20188000477E54E05A95F1F708BB17BB48BB8ACF20916F00309170002D3B3441B8F421E0AC
:2018A00020937100F894E0916F00F09170000C0120935700E8951124789480916F00909131
:2018C000700002969093700080936F00089580917100882309F43CC080916F009091700017
:2018E000813C944108F034C0F89480916F00909170008238944110F121E080917200909198
:2019000073008F559A409F70906CEEEBF4E10C0120935700E895112480917A0090917B00ED
:201920008C559A409F70906CECEBF4E10C0120935700E8951124789420936E00E0916F005F
:20194000F0917000329785E080935700E8957894109271000895FF920F931F93CF93DF930C
:2019600080910E01835087FD4EC190910B01ACE0B0E0A91BB109AE5EBE4F31E030936200CB
:2019800090910A019D3209F0FBC0883009F039C183EC8093FE008AE5809360001092F200F7
:2019A0008C91807609F478C010926C0010926B0010926A0011962C911197213009F4C5C1D8
:2019C000263009F447C0273009F042C03093670083EF90E090930D0180930C0113969C9128
:2019E00013979093F5001092F60012968C911297803379F49111ABC11496EC911497F0E04F
:201A0000EE0FFF1F81E280935700E491E093F6009EC18C3A89F4903809F099C114968C917C
:201A20001497811194C115968C91159781118FC181E0809363008BC18C3409F088C11596EE
:201A40008C911597811183C181E0809366007FC1283019F4309367007CC114968D919C910C
:201A600015979093700080936F0016968C9116978093FB00822F8950843008F06AC18FE74A
:201A800088BD309368002093FC002A3009F458C181E08093670054C112969C9112971092A7
:201AA000070111968C911197811106C01092080187E091E022E04CC0853019F490930F01D4
:201AC0003DC0863091F513968C911397813019F480EF94E104C0823041F48EED94E19093FD
:201AE0000D0180930C0122E11CC08330C9F4911108C084E295E190930D0180930C0124E0CE
:201B000010C0913019F482E195E1E9CF923041F482E095E190930D0180930C0120E101C0B4
:201B200020E080E48093F2001EC0883059F0893019F49093110102C08A3039F087E091E0E5
:201B400020E006C081E191E002C087E091E021E090930D0180930C0106C016962C9180E869
:201B60008093F2000AC017968C911797811105C016968C91821708F4282F2093610041C0FD
:201B80009091F20097FF3DC09091FB00182F981708F4192F092F011B0093FB00109267005E
:201BA0008091FC008C3019F4002349F12AC08A30D9F7FA2ECA2FDB2F1DC080916F009091D5
:201BC00070008034910590F421E020936D00FC01EE0FFF1FEE58FF4F288139813183208340
:201BE00002969093700080936F0003C0888199814FDE22968C2F8F198117F8F2D5CF109242
:201C0000610010920E018091600084FF80C0809161008F3F09F47BC0182F893008F018E016
:201C2000811B809361008091FE0098E889278093FE00112309F45AC08091F20087FF38C078
:201C40008091FB00811708F4182F811B8093FB003091FC00E0916F00F091700020E0AFEFC7
:201C6000B0E01FC03B3009F476C03930D9F7E034F10560F4EF01CC0FDD1FCE58DF4F88819C
:201C800099818D939D9332962E5F0BC0EC3B84E1F80710F08FEF01C084918C93119631964E
:201CA0002F5F2117F8F2F0937000E0936F001CC0E0910C01F0910D01AFEFB0E086FF09C03A
:201CC00084918D9331968FEF90E0810F8A13F8CF07C081918D938FEF90E0810F8A13F9CF4A
:201CE000F0930D01E0930C01193058F4612F8FEF90E05DDC1C5F1C3041F08FEF809361009D
:201D000004C08FEF809361001EE11093600084E196B3987131F48150D9F710920F0110923A
:201D20000901C1E08111C0E08091FD008C17A1F0C11103C0F8940FD17894C093FD000CC05B
:201D40008C9187FD0ACF2FEF0ACF21E00CCF24E00ACF20E008CFFFCFDF91CF911F910F9194
:201D6000FF900895C1B7B99A83E28ABD81E083BF8BB780628BBFAC9ABB9A2FE132E18AE087
:201D8000215030408040E1F700C00000BB987894E2DD80916300882321F182E090E09093C6
:201DA00065008093640013C0CF018F739927892B21F483E080935700E895CDDD80916400B0
:201DC0009091650002969093650080936400E0916400F0916500E03C94E1F90728F31092DD
:201DE000630080916600882329F0B5DD70DD10926600B1DD80916200882341F08091670009
:201E0000811104C0809168008111C2CF80916200882371F08091690081110AC088B5805F5F
:201E200088BD88B5811104C08AB590E189278ABD809169008F5F809369008EEC90E00197BD
:201E4000F1F780916A0090916B00019690936B0080936A0020916C00009711F42F5F00C0EA
:201E600020936C0030916200311105C081323EE4930708F05BC030916700332321F0813156
:201E8000974208F053C080916200882309F480CF8091680081117CCF233008F047C078CF05
:201EA00080916E0081114AC08CEB94E19093700080936F0081E08093710009DD3FC0DF015C
:201EC000AA0FBB1FAE58BF4F8D919C91309719F0E430F10531F4E054FB4E85919491805A7F
:201EE000954FD6DCE0916F00F0917000E034F10530F3EDDC10925F0217BA13BE1ABC03C047
:201F000081B78F5F81BF81B78C17D0F303C081B7815081BF81B7C817D0F391E080E80FB639
:201F2000F89486BD96BD0FBECACA13C01BBE15BAF89480916D008111B3CFDCCFE0E0F0E04A
:201F400083E080935700E8951092700010926F00C9CF80E090E0FF920F931F93CF93DF93F3
:201F600090E080E80FB6F89486BD96BD0FBEC8E0D0E010E000E8F12EF00EF1BE1CDB84332B
:201F800029E092070CF41F2D06952197A1F7212F215021BFEC01012F10C00DDB8453994042
:201FA00097FF03C09195819591098C179D0714F401B7EC0181B78F5F81BF81B790E0212FA0
:201FC00030E02F5F3F4F281739073CF701BFDF91CF911F910F91FF900895F894FFCF5AFF64
:00000001FF
